:107800000C94283C0C94433C0C94433C0C94433C17
:107810000C94433C0C94433C0C94433C0C94433CEC
:107820000C94433C0C94433C0C94433C0C94433CDC
:107830000C94433C0C94433C0C94433C0C94433CCC
:107840000C94433C0C94433C0C94433C0C94433CBC
:1078500011241FBECFE5D8E0DEBFCDBF10E0A0E60B
:10786000B0E0E8E1FFE702C005900D92A436B10751
:10787000D9F711E0A4E6B0E001C01D92A63AB10725
:10788000E1F70C944F3F0C94003C0F92AF93BF93E1
:10789000CF93DF93EF93FF93FC01EA01DB01C895DF
:1078A000099231961197D9F7FF91EF91DF91CF911E
:1078B000BF91AF910F9008950F921F920F93AF93C6
:1078C000BF93CF93DF93EF93FF93FC01EA01DB01BA
:1078D0000990199001E043D032961297C9F7FC0144
:1078E00003E03DD005E03BD0FF91EF91DF91CF91D8
:1078F000BF91AF910F911F900F9008950F931F9319
:10790000EF93FF93FC0103E02AD000E810E0E00FC2
:10791000F11FE617F707B9F7FF91EF911F910F914C
:1079200008950F930F9222D0082E09E018D00F90DF
:107930000F9108950F930F92EF93FF9317D0FC01CF
:1079400060935700C895802DFF91EF910F900F9194
:1079500008950F930BD001E102D00F910895E199A2
:10796000FECF00935700E895FFFF000000915700FD
:1079700000FDFCCF089583E089B98AB188618AB996
:1079800008958AB1877E8AB908958CB95E9BFECF2F
:107990005E9A08958CB1992708958BB199278078C4
:1079A00090700895EF92FF920F931F93CF93DF9300
:1079B0007B01C0E0D0E0C617D70770F48C010E94AD
:1079C000CD3C8823E1F30E94CA3CF80181938F01EA
:1079D0002196CE15DF0598F381E090E0DF91CF91FD
:1079E0001F910F91FF90EF900895EF92FF920F93E8
:1079F0001F93CF93DF937C018B01C0E0D0E0C017D1
:107A0000D10738F4F70181917F010E94C53C21968E
:107A1000F6CF81E090E0DF91CF911F910F91FF9021
:107A2000EF900895EF92FF920F931F93CF93DF9300
:107A30007C0100E010E00817190788F4C0E0D0E0EE
:107A400000000E94CD3C882351F4219683E0CB3680
:107A5000D807B0F30F5F1F4F0E151F0578F3DF91A6
:107A6000CF911F910F91FF90EF9008950E94C13C1C
:107A70000E9400000895DF92EF92FF920F931F93F0
:107A8000CF93DF93CDB7DEB72197DEBFCDBF8C019B
:107A90007B011982D98061E070E0CE01860F971FCB
:107AA0000E94D23C89818B31B1F761E070E0C8015E
:107AB0000E94D23C61E070E0CE01860F971F0E94C9
:107AC000D23C89819927182F002761E070E0CE0110
:107AD000860F971F0E94D23C8981080F111D61E01B
:107AE00070E0CE01860F971F0E94D23C89818E30B4
:107AF000B9F4C8010196BC01C7010E94D23C9801AB
:107B00008FEF0F3F180779F0F70181917F01D82699
:107B100021503040FFEF2F3F3F07B1F7DD2019F034
:107B200080E090E001C0C8012196DEBFCDBFDF91AB
:107B3000CF911F910F91FF90EF90DF900895CF921A
:107B4000DF92FF920F931F93CF93DF93182FEB01D8
:107B50006A018BE10E94C53C4BE1F42E812F0E940B
:107B6000C53CF1260D2F1127802F0E94C53CF02621
:107B70008C2F0E94C53CFC268EE00E94C53C8EE006
:107B8000F82621978FEFCF3FD80759F0F601819162
:107B90006F01F8260E94C53C2197FFEFCF3FDF071A
:107BA000A9F78F2D0E94C53CDF91CF911F910F91B6
:107BB000FF90DF90CF90089599278139910559F072
:107BC0008239910524F48039910529F008C0823961
:107BD000910519F004C082E003C087E001C080EC89
:107BE00099270895BF92CF92DF92EF92FF920F9361
:107BF0001F93CF93DF93B82E8B01FB018081C82F99
:107C0000DD27C231D10509F46DC0C331D105DCF4E3
:107C1000C330D10509F44DC0C430D10544F4C1309E
:107C2000D10579F1C230D10509F44AC004C1C6308A
:107C3000D10509F44AC0C630D1050CF4FCC06097E8
:107C40000CF4F9C055C0C531D10509F4C8C0C6311E
:107C5000D10544F4C331D10509F472C0649709F425
:107C60004AC0E9C0CA31D10509F4D7C0CB31D1052A
:107C700024F4669709F49AC0DEC06B9709F4C4C077
:107C8000DAC0FB01118288E0828381E4838386E588
:107C9000848382E5858389E4868383E5878380E521
:107CA00080878FE5818782E38287AB016BE070E09C
:107CB000C8C0FB0181810E94DC3DF801828301C0C4
:107CC000FB011182A801BE01BCC0FB018381992781
:107CD000982F88272481820F911D9093A50180936E
:107CE000A40107C060E070E480E090E00E947E3C68
:107CF000F8011182A3C0FB0181819927D82FCC27DD
:107D000082819927C82BD92B1182CB010296209111
:107D1000A4013091A501AC01BE01C901880F991FD2
:107D20000E94453CF801EC0FFD1F12829E01369522
:107D300027958091A4019091A501820F931F49C0BE
:107D4000FB0181819927D82FCC2782819927C82BC5
:107D5000D92BCC24DD24CC16DD06D8F4FAE0EF2EA6
:107D6000F12CE60EF71E8091A4019091A501880FD9
:107D7000991FA70160E870E08C0D9D1D0E945C3C7E
:107D800080E890E0C80ED91EE80EF91ECC16DD067C
:107D900050F30E94A93CF8011182D695C7958091B5
:107DA000A4019091A5018C0F9D1F29C0FB01818129
:107DB0009927D82FCC2782819927C82BD92B1182BC
:107DC000EC0FFD1F12828091A4019091A5018C0FF0
:107DD0009D1F9093A5018093A401239673CFFB016F
:107DE00081819927382F222782819927282B392BA7
:107DF00011828091A4019091A501820F931F90930D
:107E0000A5018093A4011AC0FB0111828481E82F8F
:107E1000FF27E05AFF4F808107C0FB01118269E014
:107E200081E090E00E949A3CF80182831382A801CD
:107E300064E070E006C089ECF8018183A80162E08B
:107E400070E08B2D0E949F3DDF91CF911F910F918C
:107E5000FF90EF90DF90CF90BF900895CF93DF9386
:107E6000CDB7DEB72197DEBFCDBF69E081E090E0FE
:107E70000E949A3C992784FF09C08F7E0E94913C02
:107E800005C064E670E089810E94F23D64E670E01E
:107E9000CE0101960E943B3D892B99F3F7CFCFE5A8
:107EA000D8E0DEBFCDBFCEE1F894AEEFB3E00E94E4
:107EB000833F802D843B71F4AFEFB3E00E94833F9A
:107EC000802D833C39F4ADEFB3E00E94833F802DD9
:107ED000992781BF0E94BB3C0E94CA3C84E690E087
:107EE0000E94123D0E94CD3C882319F00E942E3F33
:107EF00004C0C150C8BBCC2389F70E94363D80E046
:107F000090E00C948B3FE199FECFBFBBAEBBE09AF3
:087F100011960DB20895FFCF98
:047F18001E950100B1
:040000030000780081
:00000001FF
